:10000000080800103101000000000000000000009E
:100010009D0200009D0200009D0200000000000003
:100020000000000000000000000000009D02000031
:100030009D020000000000009D0200009D020000E3
:100040009D0200009D0200009D0200009D02000034
:100050009D0200009D0200009D0200009D02000024
:100060009D0200009D0200009D0200009D02000014
:100070009D0200009D0200009D0200009D02000004
:100080009D0200009D0200009D0200009D020000F4
:100090009D0200009D0200009D0200009D020000E4
:1000A0009D0200009D0200009D0200009D020000D4
:1000B0009D0200009D0200009D0200009D020000C4
:1000C0009D02000030B4174D174AD5F8C410174BE5
:1000D00041F40044C5F8C4401068154640F480213E
:1000E00011606C69002244F4802068611A60511C20
:1000F000D01C941C0432B2F1807F19601C6018601F
:10010000F4D16C69002224F4802068611A60511CCB
:10011000D01C941C0432B2F1807F19601C601860FE
:10012000F4D1DEE700C00F4020C00920000000101D
:10013000684620F007018D46F1B500F0B1F84F4850
:100140004F49884235D04F4CA14232D2024652F834
:10015000046B0B46CD4343F8046B6519A342C5F30A
:10016000810526D29DB1012D0BD0022D05D0156839
:1001700000F108021D6001F1080352F8040B43F876
:10018000040B52F8041B43F8041BA34211D29646F9
:100190005EF8047B5668D568DEF804009C464CF88F
:1001A000047B5E60CCF80400DD6010331032A342A3
:1001B000EDD335483549884234D0354CA14231D24F
:1001C000024652F8046B0B46CD4343F8046B6519A5
:1001D000A342C5F3810525D29DB1012D0BD0022D7F
:1001E00005D0156800F108021D6001F1080352F8FE
:1001F000040B43F8040B52F8041B43F8041BA342FE
:1002000010D294465CF8047B5668D568DCF804008C
:10021000194641F8047B5E604860DD60103310329F
:10022000A342EED31B491C48814221D200220B4637
:10023000CC4343F8042B04198342C4F3810417D23E
:1002400064B1012C06D0022C1CBF1A6001F1080316
:1002500043F8042B43F8042B834209D29E464EF800
:10026000042B5A60CEF80420DA6010338342F5D3B1
:10027000FFF728FFBDE8F14085467047880300007E
:1002800000000010000000108803000000000010B3
:10029000000000100000001004000010FEE700BF86
:1002A0003649202330B4C1F8A031D1F8A001334A37
:1002B00010F0400FF9D0324D0124AA20552303211C
:1002C000C2F80411C2F80C411146C2F88450C2F8B9
:1002D0008C00C2F88C30C2F88040C2F88C00C2F8A2
:1002E0008C30D1F88830254A13F0806FF9D0032183
:1002F000AA245520C2F88010C2F88C401146C2F8DA
:100300008C00D1F888301D4A13F0407FF9D02324A7
:10031000C2F8A440AA2055230124C2F8AC0011461B
:10032000C2F8AC30C2F8A040C2F8AC00C2F8AC30A1
:10033000D1F8A830114A13F4806FF9D00321AA2311
:100340005520C2F8A010C2F8AC301146C2F8AC007B
:10035000D1F8A800094A10F4407FF9D009490020DB
:1003600043F23A03C2F8A801C2F8AC01C2F8C410C3
:10037000C2F8C801136030BC704700BF00C00F4016
:0803800063000500DE8728047C
:00000001FF
